S00C0000746573742E7372656358
S11300000CC026C025C024C023C022C021C020C0EB
S11300101FC01EC01DC01CC01BC011241FBECFE5C5
S1130020D2E0DEBFCDBF10E0A0E6B0E0E2EAF0E04F
S113003003C0C89531960D92A036B107D1F710E0F0
S1130040A0E6B0E001C01D92A036B107E1F714C0EC
S1130050D7CF20E030E040E050E0261737074807CC
S113006059074CF42F5F3F4F4F4F5F4F2617370709
S113007048075907BCF30895CFE5D2E0DEBFCDBFF2
S11300808FEF87BB11BA282F80B3922F981B892F2B
S1130090880F8150992309F4892F922F981B98BBBC
S10500A0F3CF98
S9030000FC
